:10000000030883168E1C72289101343087008312F6
:100010008B0118309F009E018316433091005030B1
:100020009F00851405148312023099008101831604
:10003000863081008312071C2028A30A5120232820
:1000400051203828A30A831207108710191F23286C
:100050006120191F2328A201A101A00181011F1401
:100060009F149F1831281F1080301E020318232868
:10007000071487143F300102031D3A28A00A8101AA
:100080003C302002031D2F28A10AA0013C30210290
:10009000031D2F28A20AA1016A202202031D2F2876
:1000A0002228871061202308A600A60AA6030319A8
:1000B0005E28871461208710612056286120A301E3
:1000C00008000330A400FF30A500A50B6528A40B91
:1000D00063280800A601871A2614071AA614A60A80
:1000E000260808008E1483128701A301A101A20132
:0600F000A00183160428A4
:02400E00B031CF
:00000001FF
